:020000040800F2
:100000000050002021020008D5230008D923000851
:10001000DD230008E1230008E523000800000000BC
:10002000000000000000000000000000E9230008BC
:10003000ED23000800000000F1230008F52300086C
:10004000251F0008251F0008251F0008251F000880
:10005000251F0008251F0008251F0008251F000870
:10006000251F0008251F0008251F0008251F000860
:10007000251F0008251F0008251F0008251F000850
:10008000251F0008251F0008251F0008251F000840
:10009000251F0008251F0008251F0008251F000830
:1000A000251F0008251F0008251F0008251F000820
:1000B000251F0008251F0008251F0008251F000810
:1000C000251F0008251F0008251F0008251F000800
:1000D000251F0008251F0008251F0008251F0008F0
:1000E000251F0008251F0008251F0008000000002C
:1000F0000000000000000000000000000000000000
:1001000000000000000000005FF808F100B583B0B7
:1001100001F0F8FE304B314A1360314A1360314B25
:10012000314A03E011681960043304322F498B42CD
:10013000F8D32A4B1A682E4B9A4204D1284B1A68DE
:100140002C4B9A4200D0FEE7234B2B4A13602B4ADC
:1001500013602B4B02E000221A600433294A9342B9
:10016000F9D3254B1B6813B9244B1B6803B1FEE779
:1001700001F0D4FE694601A801F0BCFE224C234BDD
:100180001C1BA410002504E01F4B53F82530984792
:100190000135AC42F8DC1E4C1E4B1C1BA410002584
:1001A00004E01B4B53F8253098470135AC42F8DC8E
:1001B0000099019802F04AF80546174C174B1C1B92
:1001C000A41004E0013C144B53F824309847002C51
:1001D000F8DC284601F08CFEBABADECA0000002026
:1001E0001000002000000020B826000814000020A5
:1001F00078563412325476981400002034020020CD
:100200001400002038020020BC020008BC020008D4
:10021000BC020008BC020008BC020008BC020008C6
:1002200008B5FFF773FF00BF00BEFEE71EF0040F26
:100230000CBFEFF30880EFF309807146124A1047B4
:1002400000BEFEE700BEFEE71EF0040F0CBFEFF39A
:100250000880EFF3098071460C4A104700BEFEE7A4
:100260001EF0040F0CBFEFF30880EFF30980714616
:10027000074A104700BEFEE700BEFEE700BEFEE7ED
:1002800000BEFEE770470000410200085D02000862
:0402900075020008EB
:10029400B82600080000002014000020B82600083A
:1002A40000000000000000001400002038020020BC
:0802B400000000000000000042
:1002BC0010B5044600F0A8FF064BA3FB00308009E4
:1002CC0000F098F8002221464FF0FF3000F050F873
:1002DC00002010BDD34D621008B5074A136843F0D7
:1002EC0010031360032000F025F80020FFF7E0FF57
:1002FC0001F0BCFF002008BD00200240024A136838
:10030C0001331360704700BF18000020014B1868C0
:10031C00704700BF1800002010B582B00190FFF7A5
:10032C00F5FF0446FFF7F2FF001B019B9842F9D33F
:10033C0002B010BD10B50446C31E042B03D9BA215C
:10034C00094801F091FF094AD36823F4E0631B04C8
:10035C001B0C240204F4E064234343F0BF6343F416
:10036C000033D36010BD00BF7C25000800ED00E019
:10037C0070B504460E4615460F2A03D9D2211A48E9
:10038C0001F072FF0F2E03D9D321174801F06CFF37
:10039C00164BDA68C2F30222C2F10701042928BF06
:1003AC000421131D062B01D9033A00E0002201237E
:1003BC0003FA01F101393140914003FA02F2013A9A
:1003CC002A400A43002C06DA04F00F041201D2B2C0
:1003DC00074B1A5570BD1201D2B204F1604404F5FA
:1003EC00614484F8002370BD7C25000800ED00E01A
:1003FC0014ED00E00138B0F1807F0AD2064B586052
:10040C00F021064A82F823100020986007221A6017
:10041C0070470120704700BF10E000E000ED00E0E5
:10042C0010B50446042805D020B14FF4DF710848FC
:10043C0001F01AFF042C05D1064A136843F004039B
:10044C00136010BD034A136823F00403136010BD3E
:10045C007C25000810E000E008B501F0E9FF08BDBC
:10046C002DE9F04383B080460F46AE4B984213D033
:10047C0003F5806398420FD003F5806398420BD04C
:10048C0003F58063984207D003F58063984203D04C
:10049C00CF21A54801F0E8FE3B881BB9D021A2482A
:1004AC0001F0E2FE7B68012B22D9112B20D0022B0C
:1004BC001ED0122B1CD09D4A934219D002F58012EB
:1004CC00934215D002F58012934211D0A2F5F81286
:1004DC0093420DD002F58012934209D002F580129E
:1004EC00934205D0032B03D0D1218F4801F0BCFEE1
:1004FC004FF000094E462BE10125B5403C682C40DD
:10050C00A54240F02481874B984513D003F58063B6
:10051C0098450FD003F5806398450BD003F58063A5
:10052C00984507D003F58063984503D0DF217E48BA
:10053C0001F09AFE7B68122B49D00CD8022B3AD0D2
:10054C0004D8002B4FD0012B1ED067E0032B60D0BA
:10055C00112B24D062E0764A934244D008D8A2F5FD
:10056C00801293423FD002F58032934256D13AE04A
:10057C00704A934237D002F58032934233D0A2F5C1
:10058C00801293424AD12EE0FB68013B022B03D927
:10059C00E721654801F068FED7F80C903EE0FB6857
:1005AC00013B022B03D9EE215F4801F05DFEFB6895
:1005BC0003F1040932E0FB68013B022B03D9F5215E
:1005CC00594801F051FEFB6803F1080926E0FB686D
:1005DC00013B022B03D9FC21534801F045FEFB687B
:1005EC0003F10C091AE0BB68022B04D940F2091183
:1005FC004D4801F039FEBB6873B1012B04D1C8F82A
:10060C0010504FF0080909E0C8F814504FF00809D1
:10061C0004E04FF0000901E04FF00409FF2C01D871
:10062C00404601E008F10400FF2C01D8B30002E0C1
:10063C00A6F108039B0001680F229A4021EA0202EE
:10064C0009FA03F3134303607B6813F0805F7ED0D9
:10065C00394B9A6942F001029A619B6903F00103DC
:10066C000193019BB1088A1C344B53F8222006F0ED
:10067C0003039B000F20984022EA0000294A904572
:10068C000DD002F5806290450BD002F5806290454A
:10069C0009D002F58062904507D1032206E00022C2
:1006AC0004E0012202E0022200E0042202FA03F339
:1006BC0003430231214A42F821307B6813F4803F16
:1006CC0005D002F5806213682343136004E01C4AD2
:1006DC00136823EA040313607B6813F4003F04D00F
:1006EC00174A53682343536004E0154A536823EABE
:1006FC00040353607B6813F4801F04D0104A936882
:10070C002343936004E00E4A936823EA0403936046
:10071C007B6813F4001F15D0094AD3681C43D460BE
:10072C0015E000BF00080140AC25000800001110C6
:10073C0000002110000031100010024000000140A8
:10074C0000040140054AD36823EA0404D46001364E
:10075C000F2E7FF6D1AE03B0BDE8F083000401404C
:10076C0070B5064615460C4621B94FF4F27108488F
:10077C0001F07AFD012D04D940F2E511044801F095
:10078C0073FD0DB1346170BD2404346170BD00BFC4
:10079C00AC25000838B504460D4621B94FF4FD715F
:1007AC00034801F061FDE1686940E16038BD00BFBC
:1007BC00AC25000830B583B0044620B94FF48771DE
:1007CC00B94801F051FD23683BB113F00F0F04D170
:1007DC0040F20F11B44801F047FD236813F0010FEC
:1007EC0000F0A380636853B1B3F5803F07D0B3F535
:1007FC00A02F04D040F21511AB4801F035FDAB4BE6
:10080C005B6803F00C03042B0AD0A84B5B6803F065
:10081C000C03082B1BD1A54B5B6813F4803F16D03F
:10082C004FF4003393FAA3F3A04B1A684FF4003340
:10083C0093FAA3F3B3FA83F303F01F0322FA03F33F
:10084C0013F0010F71D06368002B6ED11BE363684A
:10085C00B3F5803F05D1954A136843F48033136098
:10086C0026E063B903F1804303F504331A6822F4DC
:10087C0080321A601A6822F480221A6018E0B3F5EC
:10088C00A02F0CD103F18043A3F53C331A6842F43A
:10089C0080221A601A6842F480321A6008E0834B96
:1008AC001A6822F480321A601A6822F480221A60C4
:1008BC006368EBB1FFF72AFD054605E0FFF726FD5F
:1008CC00401B642800F2E1824FF4003393FAA3F347
:1008DC00764B1A684FF4003393FAA3F3B3FA83F30D
:1008EC0003F01F0322FA03F313F0010FE6D01CE010
:1008FC00FFF70CFD054605E0FFF708FD401B6428DB
:10090C0000F2C5824FF4003393FAA3F3674B1A68D5
:10091C004FF4003393FAA3F3B3FA83F303F01F03FA
:10092C0022FA03F313F0010FE6D1236813F0020F40
:10093C0000F0A0802369012B04D940F249115A48D8
:10094C0001F092FC63691F2B04D94FF4A571564832
:10095C0001F08AFC554B5B6813F00C0F0AD0534B1B
:10096C005B6803F00C03082B27D1504B5B6813F426
:10097C00803F22D1022393FAA3F34C4B1A68022333
:10098C0093FAA3F3B3FA83F303F01F0322FA03F3EE
:10099C0013F0010F03D02369012B40F07A824348F6
:1009AC00036823F0F8016369F82292FAA2F2B2FA12
:1009BC0082F293400B4303605CE023699BB30122FA
:1009CC0092FAA2F3B3FA83F39B0003F1844303F589
:1009DC0084031A60FFF79AFC054605E0FFF796FCC6
:1009EC00401B022800F25782022393FAA3F32F4BE9
:1009FC001A68022393FAA3F3B3FA83F303F01F03E9
:100A0C0022FA03F313F0010FE8D02848036823F00F
:100A1C00F8016369F82292FAA2F2B2FA82F29340D8
:100A2C000B43036026E0012393FAA3F3B3FA83F399
:100A3C009B0003F1844303F5840300221A60FFF743
:100A4C0065FC054605E0FFF761FC401B022800F23F
:100A5C002482022393FAA3F3144B1A68022393FA09
:100A6C00A3F3B3FA83F303F01F0322FA03F313F097
:100A7C00010FE8D1236813F0080F5CD0A369012B98
:100A8C0004D94FF4C571084801F0EEFBA3696BB3B0
:100A9C00012292FAA2F3B3FA83F3054941F8232019
:100AAC00FFF734FC05460BE0F0250008001002406F
:100ABC0080044242FFF72AFC401B022800F2EF811F
:100ACC00022393FAA3F293FAA3F2A44A526A93FA7A
:100ADC00A3F3B3FA83F303F01F0322FA03F313F027
:100AEC00010FE7D00120FFF717FC24E0012393FA54
:100AFC00A3F3B3FA83F30021994A42F82310FFF7CA
:100B0C0005FC054605E0FFF701FC401B022800F23E
:100B1C00C881022393FAA3F293FAA3F28F4A526A82
:100B2C0093FAA3F3B3FA83F303F01F0322FA03F34C
:100B3C0013F0010FE7D1236813F0040F00F0AB8022
:100B4C00E368012B06D9052B04D040F2B711854878
:100B5C0001F08AFB814BDA6942F08052DA61DB6981
:100B6C0003F080530193019B7F4A136843F4807315
:100B7C001360FFF7CBFB054605E0FFF7C7FB401BF7
:100B8C00642800F29081784B1B6813F4807FF4D0BA
:100B9C00E368012B05D1714A136A43F00103136218
:100BAC0022E063B903F1804303F504331A6A22F09F
:100BBC0001021A621A6A22F004021A6214E0052B6E
:100BCC0009D1664B1A6A42F004021A621A6A42F0A0
:100BDC0001021A6208E0614B1A6A22F001021A62E1
:100BEC001A6A22F004021A62E36853B3FFF78EFB11
:100BFC00054607E0FFF78AFB401B41F28833984219
:100C0C0000F25381022393FAA3F293FAA3F3B3FAFB
:100C1C0083F35B0943F00203DBB2022B02D14F4B8F
:100C2C001A6A01E04D4B5A6A022393FAA3F3B3FA02
:100C3C0083F303F01F0322FA03F313F0010FD9D04F
:100C4C0029E0FFF763FB054607E0FFF75FFB401B5E
:100C5C0041F28833984200F22A81022393FAA3F2DC
:100C6C0093FAA3F3B3FA83F35B0943F00203DBB209
:100C7C00022B02D1394B1A6A01E0384B5A6A022313
:100C8C0093FAA3F3B3FA83F303F01F0322FA03F3EB
:100C9C0013F0010FD9D1E369022B04D940F247219B
:100CAC00304801F0E1FAE369002B00F002812B4A95
:100CBC00526802F00C02082A00F0FD80022B40F072
:100CCC00B780236A3BB1B3F5803F04D04FF4147165
:100CDC00244801F0C9FA636A73B3B3F5802F2BD0A3
:100CEC00B3F5002F28D0B3F5402F25D0B3F5801FD6
:100CFC0022D0B3F5A01F1FD0B3F5C01F1CD0B3F585
:100D0C00E01F19D0B3F5001F16D0B3F5101F13D088
:100D1C00B3F5201F10D0B3F5301F0DD0B3F5401F25
:100D2C000AD0B3F5501F07D0B3F5601F04D040F2C2
:100D3C0051210C4801F098FA4FF0807393FAA3F309
:100D4C00B3FA83F39B0003F1844303F5840300227D
:100D5C001A60FFF7DBFA05460EE000BF00100240F8
:100D6C0080044242F025000800700040FFF7CEFAE4
:100D7C00401B022800F2A1804FF0007393FAA3F3FA
:100D8C00514B1A684FF0007393FAA3F3B3FA83F341
:100D9C0003F01F0322FA03F313F0010FE6D1236AC9
:100DAC00B3F5803F10D1A3683BB1B3F5003F04D03D
:100DBC0040F26721454801F057FA43494B6823F448
:100DCC000032A36813434B603F48436823F474110B
:100DDC00236A626A13430B4343604FF0807393FAA8
:100DEC00A3F3B3FA83F39B0003F1844303F5840369
:100DFC0001221A60FFF78AFA044604E0FFF786FA2C
:100E0C00001B02285BD84FF0007393FAA3F32E4B10
:100E1C001A684FF0007393FAA3F3B3FA83F303F059
:100E2C001F0322FA03F313F0010FE7D0002049E06F
:100E3C004FF0807393FAA3F3B3FA83F39B0003F19F
:100E4C00844303F5840300221A60FFF75FFA04461B
:100E5C0004E0FFF75BFA001B022832D84FF0007356
:100E6C0093FAA3F3184B1A684FF0007393FAA3F399
:100E7C00B3FA83F303F01F0322FA03F313F0010F09
:100E8C00E7D100201EE001201CE003201AE0032023
:100E9C0018E0012016E0032014E0032012E00320E8
:100EAC0010E003200EE003200CE003200AE00320F6
:100EBC0008E0002006E0012004E0032002E003200B
:100ECC0000E0032003B030BD00100240F025000804
:100EDC0030B486B01F4D02AC28686968AA68EB680C
:100EEC000FC42B8AADF804301B4B5B6803F00C026B
:100EFC00082A2AD103F470114FF4701292FAA2F25C
:100F0C00B2FA82F221FA02F206A90A4412F8102C63
:100F1C0013F4803F15D0104B5B6803F400314FF491
:100F2C00003393FAA3F3B3FA83F321FA03F306A97C
:100F3C000B4413F8140C094BB3FBF0F000FB02F05C
:100F4C0004E0074800FB02F000E0044806B030BCA7
:100F5C00704700BFDC2500080010024000127A0028
:100F6C0000093D0070B50D46044620B94FF42F71B1
:100F7C00A04801F079F9236813F00F0F04D140F267
:100F8C00BD219C4801F070F9022D04D940F2BE211C
:100F9C00984801F069F9984B1B6803F007039D42D0
:100FAC000BD9954A136823F007032B43136013687E
:100FBC0003F007039D4240F00D81236813F0020FEC
:100FCC001DD0A368A3B1802B12D0902B10D0A02BD6
:100FDC000ED0B02B0CD0C02B0AD0D02B08D0E02BCD
:100FEC0006D0F02B04D040F2D721824801F03CF916
:100FFC0082494B6823F0F002A36813434B602368CB
:10100C0013F0010F00F081806368022B04D940F2C9
:10101C00DE21784801F028F96268012A13D14FF4D7
:10102C00003393FAA3F3754B19684FF4003393FA1A
:10103C00A3F3B3FA83F303F01F0321FA03F313F0C2
:10104C00010F28D1C8E0022A13D14FF0007393FA94
:10105C00A3F36A4B19684FF0007393FAA3F3B3FA36
:10106C0083F303F01F0321FA03F313F0010F12D1E2
:10107C00B4E0022393FAA3F3604B1968022393FAAA
:10108C00A3F3B3FA83F303F01F0321FA03F313F072
:10109C00010F00F0A58059494B6823F0030313435B
:1010AC004B60FFF733F906466368012B0FD107E05D
:1010BC00FFF72CF9801B41F28833984200F29280A2
:1010CC004E4B5B6803F00C03042BF1D11DE0022B9B
:1010DC0016D107E0FFF71AF9801B41F288339842CA
:1010EC0000F28280454B5B6803F00C03082BF1D1B6
:1010FC000BE0FFF70BF9801B41F28833984275D84F
:10110C003E4B5B6813F00C0FF3D13B4B1B6803F0A9
:10111C0007039D420AD2384A136823F007032B4376
:10112C001360136803F007039D4261D1236813F029
:10113C00040F19D0E36883B1B3F5806F0DD0B3F50C
:10114C00A06F0AD0B3F5C06F07D0B3F5E06F04D031
:10115C0040F23231274801F087F828494B6823F4D4
:10116C00E062E36813434B60236813F0080F1AD056
:10117C00236983B1B3F5806F0DD0B3F5A06F0AD09E
:10118C00B3F5C06F07D0B3F5E06F04D040F239313E
:10119C00184801F069F8194A536823F4605321691F
:1011AC0043EAC1035360FFF793FE144B5B6803F0F3
:1011BC00F002F02393FAA3F3B3FA83F322FA03F3C6
:1011CC000F4AD35CD8400F4B18600020FFF770F823
:1011DC00002070BD012070BD012070BD012070BDCC
:1011EC00012070BD032070BD032070BD032070BDB5
:1011FC00012070BDF02500080020024000100240C4
:10120C00A82600080C000020014B1868704700BF8E
:10121C000C000020002800F0B88010B504460368CC
:10122C005B4A934207D0A2F57842934203D06B21DC
:10123C00584801F019F8636833B1B3F5827F03D0D5
:10124C006C21544801F010F8A3684BB1B3F5806FD2
:10125C0006D0B3F5004F03D06D214E4801F004F8D1
:10126C00E368B3F5006F04D01BB16E21494800F060
:10127C00FBFF23692BB1022B03D06F21454800F0F3
:10128C00F3FF6369012B03D97021424800F0ECFF96
:10129C00A369B3F5007F07D033B1B3F5802F03D02A
:1012AC0071213C4800F0E0FFE3698BB1082B0FD0B3
:1012BC00102B0DD0182B0BD0202B09D0282B07D09E
:1012CC00302B05D0382B03D07221324800F0CCFFE4
:1012DC00236A2BB1802B03D073212E4800F0C4FF5E
:1012EC00636A1BB174212B4800F0BEFFA36A33B1B3
:1012FC00B3F5005F03D07521264800F0B5FFE36A13
:10130C00013B4FF6FE72934203D97621214800F03F
:10131C00ABFF94F8513013F0FF0F02D1204600F0D0
:10132C00EDFF022384F851302268136823F0400348
:10133C00136021686268A3681A43E3681A4323693F
:10134C001A4363691A43A36903F400731343E269F4
:10135C001343226A1343A26A1A430A602168638BFF
:10136C0003F00402636A13434B602368E26A1A6158
:10137C002268D36923F40063D3610020064B1870F4
:10138C006065012384F8513010BD0120704700BF07
:10139C00003001401C2600081C00002010B4036A19
:1013AC00046A24F001040462846924F0F00444EA21
:1013BC00021223F00A0319438261016210BC7047C8
:1013CC0010B4036A23F0100303628469036A24F4E3
:1013DC00704444EA023223F0A00343EA0111826113
:1013EC00016210BC704700BF836823F0700341F0AA
:1013FC00070119438160704710B4846824F47F445A
:10140C0042EA0323194344EA0103836010BC70478A
:10141C002DE9F04104460D46036A23F001030362F3
:10142C00066AD0F80480876927F073030F681F439E
:10143C0026F002038E681E431C4B98420ED1CB68DB
:10144C0033B1082B04D041F21521194800F00CFFE0
:10145C0026F00806EB681E4326F00406134B9C424C
:10146C001BD1AB69B3F5007F05D023B141F222212A
:10147C000F4800F0F9FE6B69B3F5807F05D023B1FE
:10148C0041F223210A4800F0EFFE28F440786B6902
:10149C0048EA0308AB6948EA0308C4F80480A7616A
:1014AC006B6863632662BDE8F08100BF002C0140CD
:1014BC004C2600082DE9F04104460E46036A23F43D
:1014CC0080730362056AD0F80480C76927F0730340
:1014DC000F681F4325F400738D6843EA05251D4BE7
:1014EC0098420FD1CB6833B1082B04D041F2AA211A
:1014FC00194800F0B9FE25F40065F36845EA0325A8
:10150C0025F48065134B9C421BD1B369B3F5007F66
:10151C0005D023B141F2B7210F4800F0A5FE736945
:10152C00B3F5807F05D023B141F2B8210A4800F011
:10153C009BFE28F44058736948EA0318B36948EADB
:10154C000318C4F80480E7617368E3632562BDE89F
:10155C00F08100BF002C01404C2600082DE9F04121
:10156C0004460F46036A23F480530362056AD0F8DD
:10157C000480C66926F4E6430E6843EA062625F481
:10158C0000538D6843EA05350C4B98420ED14B69DC
:10159C00B3F5807F05D023B141F2F521084800F066
:1015AC0063FE28F480487B6948EA8318C4F80480F9
:1015BC00E6617B6823642562BDE8F081002C014064
:1015CC004C260008704700BF38B590F83830012B16
:1015DC0000F005820D460446012380F838300223C2
:1015EC0080F839300B68B3F5805F16D0B3F5005F27
:1015FC0013D093B1102B10D0202B0ED0302B0CD03D
:10160C00402B0AD0502B08D0602B06D0702B04D066
:10161C0040F64B71A04800F027FE2268936823F433
:10162C007F4323F0770393602B68402B00F03881C5
:10163C000ED8102B00F0828103D8002B00F06581AE
:10164C00C6E1202B00F09381302B00F0A981BFE183
:10165C00702B28D006D8502B00F0B380602B00F0F4
:10166C00E580B5E1B3F5805F03D0B3F5005F61D0E1
:10167C00AEE12368894A93420FD0B3F1804F0CD06E
:10168C00A2F59432934208D002F58062934204D0C2
:10169C0040F65771804800F0E7FD2268936823F00C
:1016AC000703936094E123687C4A93420FD0B3F113
:1016BC00804F0CD0A2F59432934208D002F5806290
:1016CC00934204D04FF47661734800F0CDFDAB68C3
:1016DC006BB1B3F5805F0AD0B3F5005F07D0B3F5FB
:1016EC00405F04D040F663716B4800F0BDFD6B6841
:1016FC00B3F5004F0AD04BB143B1022B06D00A2BE5
:10170C0004D040F66471644800F0AEFDEB680F2B1A
:10171C0004D940F66571604800F0A6FDEB686A6874
:10172C00A9682068FFF768FE2268936843F0770386
:10173C0093604DE12368594A93420FD0B3F1804F27
:10174C000CD0A2F59432934208D002F580629342F9
:10175C0004D040F67A71504800F086FDAB686BB14E
:10176C00B3F5805F0AD0B3F5005F07D0B3F5405FE7
:10177C0004D040F67D71484800F076FD6B68B3F5F7
:10178C00004F0AD04BB143B1022B06D00A2B04D028
:10179C0040F67E71404800F067FDEB680F2B04D9D2
:1017AC0040F67F713C4800F05FFDEB686A68A96801
:1017BC002068FFF721FE2268936843F4804393600E
:1017CC0006E12368354A93420FD0B3F1804F0CD019
:1017DC00A2F59432934208D002F58062934204D071
:1017EC0040F68E712C4800F03FFD6B68B3F5004F4E
:1017FC000AD04BB143B1022B06D00A2B04D040F6D1
:10180C009171254800F030FDEB680F2B04D940F6A0
:10181C009271214800F028FDEA6869682068FFF79A
:10182C00BDFD50212068FFF7DFFDD1E023681B4A86
:10183C0093420FD0B3F1804F0CD0A2F59432934267
:10184C0008D002F58062934204D040F69D71124894
:10185C0000F00AFD6B68B3F5004F0AD04BB143B1F1
:10186C00022B06D00A2B04D04FF47A610A4800F000
:10187C00FBFCEB680F2B04D940F6A171064800F075
:10188C00F3FCEA6869682068FFF79AFD602120681C
:10189C00FFF7AAFD9CE000BF4C260008002C01407D
:1018AC002368504A93420FD0B3F1804F0CD0A2F56D
:1018BC009432934208D002F58062934204D040F6F1
:1018CC00AC71494800F0D0FC6B68B3F5004F0AD0FE
:1018DC004BB143B1022B06D00A2B04D040F6AF71AA
:1018EC00414800F0C1FCEB680F2B04D94FF47B612D
:1018FC003D4800F0B9FCEA6869682068FFF74EFDC6
:10190C0040212068FFF770FD62E02368354A93425E
:10191C000FD0B3F1804F0CD0A2F59432934208D083
:10192C0002F58062934204D040F6BB712E4800F061
:10193C009BFC00212068FFF757FD49E02368294AEA
:10194C0093420FD0B3F1804F0CD0A2F59432934256
:10195C0008D002F58062934204D040F6C37122484D
:10196C0000F082FC10212068FFF73EFD30E0236878
:10197C001C4A93420FD0B3F1804F0CD0A2F5943295
:10198C00934208D002F58062934204D040F6CB71AA
:10199C00154800F069FC20212068FFF725FD17E0B1
:1019AC002368104A93420FD0B3F1804F0CD0A2F5AC
:1019BC009432934208D002F58062934204D040F6F0
:1019CC00D371094800F050FC30212068FFF70CFD62
:1019DC00012384F83930002084F8380038BD022007
:1019EC0038BD00BF002C01404C2600080368184A83
:1019FC0090420AD0B0F1804F07D0A2F594329042B9
:101A0C0003D002F58062904203D123F070034A6840
:101A1C0013430F4A90420AD0B0F1804F07D0A2F581
:101A2C009432904203D002F58062904203D123F4A9
:101A3C004073CA68134303608B68C3620B6883628C
:101A4C00034B984201D10B69036301234361704737
:101A5C00002C0140002845D010B504460368224AEA
:101A6C0093420ED0B3F1804F0BD0A2F59432934237
:101A7C0007D002F58062934203D0D7211B4800F0B7
:101A8C00F3FBA3685BB1102B09D0202B07D0402BA4
:101A9C0005D0602B03D0D821144800F0E5FB236956
:101AAC004BB1B3F5807F06D0B3F5007F03D0D921BD
:101ABC000E4800F0D9FB94F8393013F0FF0F05D124
:101ACC00002384F83830204600F044FC022384F8CC
:101ADC003930211D2068FFF789FF012384F8393044
:101AEC00002010BD01207047002C01404C2600083E
:101AFC00002848D010B504460368244A93420FD0FE
:101B0C00B3F1804F0CD0A2F59432934208D002F579
:101B1C008062934204D040F2E2311D4800F0A4FBF5
:101B2C00A36863B1102B0AD0202B08D0402B06D011
:101B3C00602B04D040F2E331154800F095FB23698B
:101B4C0053B1B3F5807F07D0B3F5007F04D04FF4C9
:101B5C0079710F4800F088FB94F8393013F0FF0FBF
:101B6C0005D1002384F838302046FFF72BFD0223E3
:101B7C0084F83930211D2068FFF738FF012384F8E1
:101B8C003930002010BD0120704700BF002C0140EF
:101B9C004C2600082DE9F04104460F46036A23F059
:101BAC0010030362056AD0F80480866926F4E643C4
:101BBC000E6843EA062625F020038D6843EA0515D6
:101BCC001C4B98420FD1CB6833B1082B04D041F297
:101BDC005F21194800F048FB25F08005FB6845EAB9
:101BEC00031525F04005134B9C421BD1BB69B3F583
:101BFC00007F05D023B141F26D210F4800F034FB7A
:101C0C007B69B3F5807F05D023B141F26E210A4880
:101C1C0000F02AFB28F440687B6948EA8308BB691A
:101C2C0048EA8308C4F80480A6617B68A363256234
:101C3C00BDE8F081002C01404C26000890F83830AB
:101C4C00012B00F0E88070B516460D4604460123C2
:101C5C0080F8383062B1042A0AD0082A08D00C2A3D
:101C6C0006D0182A04D040F60D416C4800F0FCFA5E
:101C7C002B68602B06D0702B04D040F60E416748C1
:101C8C0000F0F2FAAB6833B1022B04D040F60F41EE
:101C9C00624800F0E9FA2B6933B1042B04D04FF4FD
:101CAC0041615E4800F0E0FA022384F839300C2ED2
:101CBC0000F2AA80DFE806F007A8A8A82FA8A8A819
:101CCC0058A8A8A880002368554A93420FD0B3F1B6
:101CDC00804F0CD0A2F59432934208D002F580626A
:101CEC00934204D040F618414C4800F0BDFA294606
:101CFC002068FFF78DFB2268936943F0080393611A
:101D0C002268936923F004039361226891692B691B
:101D1C000B43936178E02368414A93420FD0B3F1AF
:101D2C00804F0CD0A2F59432934208D002F5806219
:101D3C00934204D040F62741384800F095FA2946E2
:101D4C002068FFF727FF2268936943F400639361CF
:101D5C002268936923F480639361226893692969EB
:101D6C0043EA012393614FE023682D4A93420FD03D
:101D7C00B3F1804F0CD0A2F59432934208D002F507
:101D8C008062934204D040F63641244800F06CFA4D
:101D9C0029462068FFF78EFB2268D36943F00803BD
:101DAC00D3612268D36923F00403D3612268D1691B
:101DBC002B690B43D36127E02368194A93420FD058
:101DCC00B3F1804F0CD0A2F59432934208D002F5B7
:101DDC008062934204D040F64541104800F044FA2A
:101DEC0029462068FFF7BAFB2268D36943F40063E5
:101DFC00D3612268D36923F48063D3612268D369E9
:101E0C00296943EA0123D361012384F83930002086
:101E1C0084F8380070BD0220704700BF4C260008C3
:101E2C00002C014038B504460D4603682B4A9342FA
:101E3C000FD0B3F1804F0CD0A2F59432934208D05E
:101E4C0002F58062934204D040F28C61244800F089
:101E5C000BFA2B6893B1102B10D0202B0ED0302BFB
:101E6C000CD0402B0AD0502B08D0602B06D0702BF6
:101E7C0004D040F28D611A4800F0F6F96B68802BA3
:101E8C0005D023B140F28E61154800F0EDF994F8BD
:101E9C003830012B1FD0012284F83820022384F81B
:101EAC00393021684B6823F070034B602168486817
:101EBC002B6803434B6021688B6823F080038B6095
:101ECC00216888686B6803438B6084F83920002094
:101EDC0084F8380038BD022038BD00BF002C01400A
:101EEC0078260008FEE700BF01230360014B0B605E
:101EFC00704700BF0400002008B500F00FF8024B3B
:101F0C00024A9A6008BD00BF00ED00E00000000826
:101F1C0008B500F029F808BDFEE700000F4B1A6861
:101F2C0042F001021A6059680D4A0A405A601A6858
:101F3C0022F0847222F480321A601A6822F4802211
:101F4C001A605A6822F4FE025A604FF41F029A601B
:101F5C004FF00062034B9A60704700BF00100240C4
:101F6C000000FFF800ED00E01F4B5B6803F00C0372
:101F7C00042B06D0082B08D03BBB1C4A1C4B1A6008
:101F8C0026E01A4A1A4B1A6022E0174A5368526824
:101F9C00C3F38343023312F4803F05D1154A02FB8D
:101FAC0003F3134A136013E00F4A526812F4003F14
:101FBC0005D0104A02FB03F30D4A136008E00B4AEC
:101FCC0002FB03F30A4A136002E0084A084B1A604A
:101FDC00054B5B68C3F30313074AD15C044A1368CF
:101FEC00CB401360704700BF0010024000127A0013
:101FFC000C00002000093D00A826000810B588B090
:10200C00174B9A6942F010029A619A6902F0100219
:10201C000192019A9A6942F020029A619A6902F03F
:10202C0020020292029A9A6942F004029A619B6918
:10203C0003F004030393039B0A4C00224FF4C041AA
:10204C002046FEF78DFB4FF4C04304930123059308
:10205C000223079304A92046FEF702FA08B010BD2C
:10206C00001002400010014008B500F0E5F9FEE751
:10207C0008B50E480E4B03604FF482734360002387
:10208C008360C36002220261012242614FF400723C
:10209C0082611822C2610362436283620A23C362B3
:1020AC00FFF7B8F808B1FFF7DFFF08BD60000020AC
:1020BC000030014000B587B01448154B0360242351
:1020CC004360002383604FF47A72C2600361436102
:1020DC00FFF7C0FC08B1FFF7C7FF06A94FF4805308
:1020EC0041F8103D0948FFF76FFA08B1FFF7BCFF44
:1020FC0000230093019369460448FFF793FE08B14F
:10210C00FFF7B2FF07B05DF804FB00BF240000200E
:10211C00002C014000B58FB02A484FF0804303607B
:10212C00002343608360C3600361FFF793FC08B135
:10213C00FFF79AFF0EA94FF4805341F8103D214848
:10214C00FFF742FA08B1FFF78FFF1E48FFF7D0FCEC
:10215C0008B1FFF789FF00230893099308A91948D0
:10216C00FFF760FE08B1FFF77FFF602301930022A9
:10217C0002920392059201A91248FFF75FFD08B184
:10218C00FFF772FF04220DEB02010E48FFF756FD1C
:10219C0008B1FFF769FF082201A90A48FFF74EFDB5
:1021AC0008B1FFF761FF0C2201A90648FFF746FDB5
:1021BC0008B1FFF759FF034800F0F0F80FB05DF8D5
:1021CC0004FB00BFB800002000B591B001230693BA
:1021DC004FF4803307930022089202220D920E9343
:1021EC004FF4E0130F9306A8FEF7E4FA08B1FFF7DB
:1021FC003BFF0F23019302210291002303934FF421
:10220C0080620492059301A8FEF7ACFE08B1FFF7BB
:10221C002BFFFEF7F9FF094BA3FB00308009FEF7FB
:10222C00E9F80420FEF7FCF8002211464FF0FF30CD
:10223C00FEF79EF811B05DF804FB00BFD34D6210A1
:10224C0008B500F0EDF8FEF747F8FFF7BDFFFFF714
:10225C00D5FEFFF70DFFFFF72DFFFFF75BFF00F03B
:10226C00F5F800F0E1F8FCE7704700BF00B583B06B
:10227C00204B9A6942F001029A619B6903F00103B9
:10228C000193019B0320FEF755F8002211466FF0D5
:10229C000B00FEF76DF8002211466FF00A00FEF7F6
:1022AC0067F8002211466FF00900FEF761F8002272
:1022BC0011466FF00400FEF75BF8002211466FF038
:1022CC000300FEF755F8002211466FF00100FEF7EF
:1022DC004FF8002211464FF0FF30FEF749F8064A3E
:1022EC00536823F0E06343F00073536003B05DF870
:1022FC0004FB00BF00100240000001400268134BB9
:10230C009A4222D110B586B003F560439A6942F423
:10231C0080529A619B6903F480530193019BA02323
:10232C0002930223039303230593094C02A920462D
:10233C00FEF796F84023029300230393049302A91B
:10234C002046FEF78DF806B010BD704700300140F6
:10235C000008014082B003680E4A93420AD10E4B2A
:10236C009A6942F400629A619B6903F400630093DA
:10237C00009B0DE0B3F1804F0AD103F50433DA6909
:10238C0042F00102DA61DB6903F001030193019B66
:10239C0002B07047002C0140001002400368B3F1FA
:1023AC00804F0DD100B585B00F230093022301930C
:1023BC00039369460348FEF753F805B05DF804FB38
:1023CC00704700BF00080140704700BFFEE700BF28
:1023DC00FEE700BFFEE700BFFEE700BF704700BF8F
:1023EC00704700BF704700BF08B5FDF787FFFEF7C9
:1023FC0033F808BD08B54FF400510248FEF7CAF98E
:10240C0008BD00BF0010014008B54FF47A730022DC
:10241C001146024800F036F808BD00BF0124000840
:10242C0008B500F017F808BD08B500F04BF808BD6A
:10243C0008B500F073F808BD08B501224FF48041CF
:10244C000148FEF78DF908BD0010014008B5FFF7F3
:10245C00DBFF08BD30B400230EE0094C9900CA180C
:10246C00950060190022625142600272C2602846D7
:10247C00204402610133DBB20F2BEED930BC704724
:10248C00F4000020F0B5002417E0274604EB840686
:10249C00B5000B4E3544ED686DB934464FEA870EE6
:1024AC000EEB0705AE00A519A2516B6000232B7231
:1024BC00E8602961F0BD0134E4B20F2CE5D9F0BD20
:1024CC00F400002070B5002422E004EB8402930099
:1024DC00114A1344DB68CBB104EB840293000E4A1F
:1024EC0013441B7A93B1A10021448A000A4E16446E
:1024FC00013B3372F36830699847736833B904EB66
:10250C008405AB00044A13440022DA600134E4B2BF
:10251C000F2CDAD970BD00BFF400002070B400237A
:10252C001FE003EB8300820010480244D268B2B172
:10253C0003EB830082000D48825852B904469A007E
:10254C00D518A80025186E682650287A411C2972C7
:10255C0005E003EB83018800013A04490A5001337A
:10256C00DBB20F2BDDD970BC704700BFF40000202C
:10257C002E2E2F73797374656D2F7372632F737492
:10258C006D3332663178782F73746D3332663178EF
:10259C00785F68616C5F636F727465782E6300009E
:1025AC002E2E2F73797374656D2F7372632F737462
:1025BC006D3332663178782F73746D3332663178BF
:1025CC00785F68616C5F6770696F2E630000000054
:1025DC0002030405060708090A0B0C0D0E0F101058
:1025EC00010200002E2E2F73797374656D2F737298
:1025FC00632F73746D3332663178782F73746D3347
:10260C0032663178785F68616C5F7263632E630049
:10261C002E2E2F73797374656D2F7372632F7374F1
:10262C006D3332663178782F73746D33326631784E
:10263C00785F68616C5F7370695F65782E6300000A
:10264C002E2E2F73797374656D2F7372632F7374C1
:10265C006D3332663178782F73746D33326631781E
:10266C00785F68616C5F74696D2E63002E2E2F731A
:10267C00797374656D2F7372632F73746D33326657
:10268C003178782F73746D3332663178785F686186
:10269C006C5F74696D5F65782E630000000000004C
:0C26AC00000000000102030406070809FA
:1026B80078563412200000200000000000A24A04CE
:0426C800325476987A
:040000050800010DE1
:00000001FF
